:100000000C945B000C9483000C9483000C9483008C
:100010000C9483000C9483000C9483000C94830054
:100020000C9483000C9483000C9483000C94830044
:100030000C9483000C9483000C9483000C94830034
:100040000C943B030C9483000C94BC050C9483002B
:100050000C9483000C9483000C9483000C94830014
:100060000C9483000C948300000024272A000025B0
:10007000282B000023262904040404040404040299
:100080000202020202030303030303010204081035
:100090002040800102040810200102040810200002
:1000A0000000070002010000030406000000000039
:1000B00000000000930111241FBECFEFD4E0DEBF8B
:1000C000CDBF11E0A0E0B1E0EAECFCE002C0059099
:1000D0000D92A431B107D9F711E0A4E1B1E001C05C
:1000E0001D92AC3BB107E1F710E0C6EBD0E004C0D5
:1000F0002297FE010E945F06C43BD107C9F70E9408
:100100008C010C9463060C9400000F931F93CF9303
:10011000DF930CE111E0C0E0D0E0C330D105F9F08D
:10012000C430D1054CF4C130D105A9F0C230D1059D
:10013000A4F4209771F03EC0C530D105C9F0C53098
:10014000D1057CF0C630D105D1F0C730D10591F58D
:1001500022C060E007C060E00CC060E011C060E059
:100160001BC061E0809102010E94AB0460E00DC001
:1001700061E0809102010E94AB0460E012C061E086
:10018000809102010E94AB0461E0809104010E9411
:10019000AB0460E00BC061E0809102010E94AB04FF
:1001A00061E0809104010E94AB0461E0809106014E
:1001B0000E94AB046AE070E080E090E00E94A60339
:1001C000809114010E941B049093170180931601E3
:1001D000F801819391938F01809108019091090119
:1001E000AC0173E0440F551F7A95E1F7880F991F12
:1001F000480F591F48535F4F4C0F5D1F662757FD2F
:100200006095762F20E030E08EE291E00E941B03A3
:10021000809116019091170165E070E00E94F90548
:10022000AB01662757FD6095762F20E030E08EE227
:1002300091E00E941B032196C830D10509F06DCFD3
:10024000809100010E941B04909317018093160176
:1002500090932D0180932C018091080190910901C8
:10026000AC0133E0440F551F3A95E1F7880F991F11
:10027000480F591F40535F4F662757FD6095762FF3
:1002800020E030E08EE291E00E941B038091160195
:100290009091170165E070E00E94F905AB016627B7
:1002A00057FD6095762F20E030E08EE291E00E94CD
:1002B0001B0364E170E080E090E00E94A603DF9100
:1002C000CF911F910F91089540E052EC61E070E0F2
:1002D0008EE291E00E94A70161E0809102010E94FC
:1002E0008D0461E0809104010E948D0461E08091A1
:1002F00006010E948D0460E08EE00E948D0460E0A3
:100300008FE00E948D0461E08EE00E94AB0461E00A
:100310008FE00E94AB0408950E94DE030E946401F6
:100320000E948500FDCF80E191E090932F018093A2
:100330002E010895862F0E947B0508950E94B30523
:1003400008950E94940508950E9483050895CB01A5
:10035000BA010E9442050895DC01ED91FC910190E3
:10036000F081E02D09950895DC01ED91FC9101905B
:10037000F081E02D099508950F931F93CF93DF939C
:100380008C01EB0109C02196D801ED91FC910190FF
:10039000F081E02DC801099568816623A1F7DF91FE
:1003A000CF911F910F9108950F931F938C01DC0142
:1003B000ED91FC910190F081E02D6DE00995D8015F
:1003C000ED91FC910190F081E02D6AE0C801099562
:1003D0001F910F9108950F931F938C01DC01ED91F4
:1003E000FC910190F081E02D0995C8010E94D40193
:1003F0001F910F9108950F931F938C010E94BC01D0
:10040000C8010E94D4011F910F9108950F931F936B
:100410008C01DC01ED91FC910190F081E02D0995BA
:10042000C8010E94D4011F910F9108952F923F920D
:100430004F925F926F927F928F929F92AF92BF92F4
:10044000CF92DF92EF92FF920F931F93DF93CF93A0
:10045000CDB7DEB7A0970FB6F894DEBF0FBECDBF05
:100460001C016A017B01411551056105710549F4C3
:10047000DC01ED91FC910190F081E02D60E30995A4
:1004800054C0882499245401422E5524662477248C
:1004900001E010E00C0F1D1F080D191DC701B6016A
:1004A000A30192010E940C06F80160830894811C4C
:1004B000911CA11CB11CC701B601A30192010E94AD
:1004C0000C06C901DA016C017D01C114D104E104FB
:1004D000F104F1F681E0E82EF12CEC0EFD1EE80CA3
:1004E000F91C3E010894611C711CD501C4010197DF
:1004F000A109B1096C01C818D90814C0F601EE0DA4
:10050000FF1D60816A3010F4605D01C0695CD1013B
:10051000ED91FC910190F081E02DC10109950894C5
:10052000E108F1086E147F0449F7A0960FB6F8941D
:10053000DEBF0FBECDBFCF91DF911F910F91FF9016
:10054000EF90DF90CF90BF90AF909F908F907F9073
:100550006F905F904F903F902F9008952AE00E94F7
:10056000160208950F931F938C010E94AE02C801DA
:100570000E94D4011F910F910895AB0160E070E0DB
:100580000E94AE0208950F931F938C01AB0160E0AF
:1005900070E00E94AE02C8010E94D4011F910F9129
:1005A0000895EF92FF920F931F93CF93DF93EC0187
:1005B0007A018B0177FF0FC0E881F9810190F0810A
:1005C000E02D6DE2099510950095F094E094E11C02
:1005D000F11C011D111D2AE0B801A701CE010E94E6
:1005E0001602DF91CF911F910F91FF90EF90089528
:1005F0000F931F938C010E94D102C8010E94D40165
:100600001F910F910895AB01662757FD6095762FD6
:100610000E94D10208950F931F938C01AB016627AE
:1006200057FD6095762F0E94D102C8010E94D40127
:100630001F910F910895DC012115310541F4ED91D1
:10064000FC910190F081E02D642F099508952A30E6
:10065000310519F40E94D10208950E9416020895EE
:100660000F931F938C010E941B03C8010E94D401A9
:100670001F910F9108951F920F920FB60F921124A0
:100680002F938F939F93AF93BF938091300190915D
:100690003101A0913201B09133018050904CAF4FA5
:1006A000BF4F8093300190933101A0933201B093FA
:1006B000330127C08091300190913101A091320126
:1006C000B091330180589E43A040B04080933001E8
:1006D00090933101A0933201B093330180913401A2
:1006E00090913501A0913601B09137010196A11D7D
:1006F000B11D8093340190933501A0933601B093DE
:1007000037018091300190913101A0913201B09177
:10071000330181589E43A040B04060F6BF91AF9135
:100720009F918F912F910F900FBE0F901F90189552
:100730008FB7F89420913401309135014091360102
:10074000509137018FBFB901CA010895EF92FF920E
:100750000F931F937B018C018FB7F8944091340164
:100760005091350160913601709137018FBF2FB7DD
:10077000F8948091340190913501A0913601B091A7
:1007800037012FBF841B950BA60BB70B8E159F054A
:10079000A007B10760F31F910F91FF90EF900895AC
:1007A000019759F0FC01EE0FFF1FEE0FFF1F32976C
:1007B0008FB7F8943197F1F78FBF0895789484B587
:1007C000826084BD84B5816084BD85B5826085BD4D
:1007D00085B5816085BDEEE6F0E080818160808333
:1007E000E1E8F0E0808182608083808181608083A5
:1007F000E0E8F0E0808181608083E1EBF0E08081DF
:1008000084608083E0EBF0E0808181608083EAE7B0
:10081000F0E0808184608083808182608083808139
:10082000816080838081806880831092C1000895F8
:100830008093120108958F70909112019295990FF3
:10084000990F907C982B90937C0080917A00806423
:1008500080937A0080917A0086FDFCCF2091780009
:1008600040917900942F80E030E0282B392BC9018A
:1008700008951F93CF93DF93182FEB0161E00E943F
:100880008D04E12FF0E0E156FF4F8491833051F465
:1008900080918000806880938000D0938900C0930D
:1008A000880037C0843051F480918000806280934A
:1008B0008000D0938B00C0938A002BC0813029F434
:1008C00084B5806884BDC7BD24C0823029F484B556
:1008D000806284BDC8BD1DC0863041F48091B000E7
:1008E00080688093B000C093B30013C0873041F498
:1008F0008091B00080628093B000C093B40009C0C2
:10090000C038D10514F460E001C061E0812F0E947D
:10091000AB04DF91CF911F910895282F30E0C901DA
:1009200085579F4FFC01949129583F4FF9018491BD
:10093000882381F0E82FF0E0E859FF4FE491F0E0E0
:10094000662329F48081909589238083089580818E
:10095000892B80830895482F50E0CA0181569F4F0C
:10096000FC012491CA0185579F4FFC01949149587D
:100970005F4FFA0134913323C1F1222331F1233047
:1009800021F4809180008F7705C0243031F480916C
:1009900080008F7D8093800018C0213019F484B5C9
:1009A0008F7704C0223021F484B58F7D84BD0DC0C3
:1009B000263021F48091B0008F7705C0273029F4CC
:1009C0008091B0008F7D8093B000E32FF0E0E35979
:1009D000FF4FE491F0E0662329F48081909589230C
:1009E000808308958081892B80830895482F50E06B
:1009F000CA0181569F4FFC012491CA0185579F4F20
:100A0000FC01949149585F4FFA013491332319F452
:100A100020E030E035C0222331F1233021F48091F1
:100A200080008F7705C0243031F4809180008F7D65
:100A30008093800018C0213019F484B58F7704C0EA
:100A4000223021F484B58F7D84BD0DC0263021F481
:100A50008091B0008F7705C0273029F48091B000D5
:100A60008F7D8093B000E32FF0E0EE58FF4FE491CC
:100A7000F0E0808120E030E0892311F021E030E0D7
:100A8000C9010895EF92FF920F931F937B018C0190
:100A900022E030E040E050E00E942E06205C3D4B1A
:100AA000404F5F4FCA01B901A80197010E942E066D
:100AB000C901DA010197A109B109292F3A2F4B2F5A
:100AC000552747FD5A950196A11DB11D2093C500DC
:100AD00081508093C400E1ECF0E0808180618083EC
:100AE0008081886080838081806880831F910F91DE
:100AF000FF90EF900895982F8091C00085FFFCCF64
:100B00009093C600089580913801909139018058E2
:100B10009F4F20913A0130913B01821B930B60E87B
:100B200070E00E94F905089540913A0150913B010F
:100B300080913801909139018417950719F42FEFAE
:100B40003FEF0FC0FA01E45CFE4F2081CA0101961D
:100B500060E870E00E94F90590933B0180933A01B0
:100B600030E0C901089580913A0190913B01909342
:100B700039018093380108951F920F920FB60F929A
:100B800011242F933F934F935F936F937F938F9392
:100B90009F93AF93BF93EF93FF934091C600E09173
:100BA0003801F0913901CF01019660E870E00E94B0
:100BB000F9059C0180913A0190913B012817390772
:100BC00039F0E45CFE4F40833093390120933801C3
:100BD000FF91EF91BF91AF919F918F917F916F9115
:100BE0005F914F913F912F910F900FBE0F901F90EB
:100BF000189597FB092E07260AD077FD04D049D017
:100C000006D000201AF4709561957F4F0895F6F78D
:100C1000909581959F4F0895A1E21A2EAA1BBB1BA8
:100C2000FD010DC0AA1FBB1FEE1FFF1FA217B307B8
:100C3000E407F50720F0A21BB30BE40BF50B661FCE
:100C4000771F881F991F1A9469F760957095809592
:100C500090959B01AC01BD01CF01089597FB092E32
:100C600005260ED057FD04D0D7DF0AD0001C38F47B
:100C700050954095309521953F4F4F4F5F4F0895C8
:100C8000F6F790958095709561957F4F8F4F9F4FA8
:100C90000895AA1BBB1B51E107C0AA1FBB1FA617C3
:100CA000B70710F0A61BB70B881F991F5A95A9F715
:100CB00080959095BC01CD010895EE0FFF1F059022
:0A0CC000F491E02D0994F894FFCFA1
:100CCA00010006000500040001000A0000000000FF
:040CDA009A0101007A
:00000001FF
